:1000000002009F53E630900006120393543FF5E739
:1000100012037A6401700343E68090000312039395
:100020006401700343E602900004120393640170BC
:100030000343E780900005120393700343E74043B6
:10004000BA80900001120393FFD3940374809480CC
:10005000500890FEAEE054FC4FF090000212039363
:10006000FFD3940174809480500EEF25E025E0FFCB
:1000700090FEAEE054FB4FF053BA7F22750801E4C6
:10008000F509750A01F50C750D01750B01750E105A
:10009000FB7A007908120003E4FD7F030203257850
:1000A0007FE4F6D8FD75810E0203F20203E1EFD37F
:1000B00094077480948040037FFF2212037AFED35A
:1000C00094037480948040037FFF22EF7044EE70AD
:1000D0000B900001120393F45293529412037A642A
:1000E00001700B9000011203934293F45294120397
:1000F0007AFE6402700A90000112039342934294C4
:10010000EE6403700D900001120393FEF45293EE1F
:100110004294EF6401704612037AFE700B90000166
:10012000120393F452915292EE6401700B9000010D
:100130001203934291F4529212037A6402700A906D
:1001400000011203934291429212037A6403700DEC
:10015000900001120393FEF45291EE4292EF64027A
:10016000704612037AFE700B900001120393F45252
:10017000955296EE6401700B900001120393429524
:10018000F4529612037A6402700A900001120393EB
:100190004295429612037A6403700D900001120397
:1001A00093FEF45295EE4296EF6403704612037A82
:1001B000FE700B900001120393F452B152B2EE6440
:1001C00001700B90000112039342B1F452B212037A
:1001D0007A6402700A90000112039342B142B21293
:1001E000037A6403700D900001120393FEF452B180
:1001F000EE42B2EF6404704612037AFE700B900078
:1002000001120393F452B352B4EE6401700B9000E8
:100210000112039342B3F452B412037A6402700AD7
:1002200090000112039342B342B412037A64037044
:100230000D900001120393FEF452B3EE42B4EF644A
:1002400005704612037AFE700B900001120393F4BE
:1002500052C952CAEE6401700B900001120393421E
:10026000C9F452CA12037A6402700A9000011203A0
:100270009342C942CA12037A6403700D90000112BE
:100280000393FEF452C9EE42CAEF640670461203AD
:100290007AFE700B900001120393F452CB52CCEE15
:1002A0006401700B90000112039342CBF452CC1204
:1002B000037A6402700A90000112039342CB42CC8D
:1002C00012037A6403700D900001120393FEF4523E
:1002D000CBEE42CCEF6407704912037AFF7E0070C8
:1002E0000B900001120393F452E152E2EF64014ECD
:1002F000700B90000112039342E1F452E212037A70
:100300006402700A90000112039342E142E2120378
:100310007A6403700D900001120393FFF452E1EF31
:1003200042E27F0022EF30E10543E620800353E6FE
:10033000DFEF30E00543E610800353E6EFEDFF7E8C
:1003400000D3940374809480502DEF700653B6DF71
:1003500053B5DFEF64014E700653B6DF43B520EFAF
:1003600064024E700643B62053B5DFEF64034E704F
:100370000643B62043B5207F0022BB010689828A4E
:1003800083E0225002E722BBFE02E32289828A83B5
:10039000E49322BB010CE58229F582E5833AF583DB
:1003A000E0225006E92582F8E622BBFE06E9258216
:1003B000F8E222E58229F582E5833AF583E4932287
:1003C0007509C07508017B007A0079087F03120067
:1003D000AE750901E4F508FB7A0079087F05020093
:1003E000AEC0E0C0D053E6BFE5E61392C8D0D0D08F
:0C03F000E0321203C012007CD2AF80FE8D
:00000001FF
